:100000000C94A3000C94CB000C94CB000C94CB006C
:100010000C94CB000C94CB000C94CB000C94CB0034
:100020000C94CB000C94BB040C94CB000C94CB0030
:100030000C94CB000C94CB000C94CB000C94CB0014
:100040000C947C150C94CB000C94AB060C94DC0641
:100050000C94CB000C94CB000C94CB000C94CB00F4
:100060000C94CB000C94CB0007634236B79BD8A707
:100070001A39685618AEBAAB558C1D3CB7CC5763CD
:10008000BD6DEDFD753EF6177231BF000000803F7B
:1000900008000000BE922449123EABAAAA2ABECD97
:1000A000CCCC4C3E00000080BEABAAAAAA3E000009
:1000B0000000BF000000803F000000000008417801
:1000C000D3BB4387D1133D190E3CC3BD4282AD2B38
:1000D0003E68EC8276BED98FE1A93E4C80EFFFBE30
:1000E00001C4FF7F3F00000000000000000024006A
:1000F00027002A0000000000250028002B00000037
:10010000000023002600290004040404040404045D
:1001100002020202020203030303030301020408B2
:100120001020408001020408102001020408102061
:1001300000000007000201000003040600000000A8
:1001400000000000370811241FBECFEFD8E0DEBF4B
:10015000CDBF12E0A0E0B1E0E8ECFCE302C0059006
:100160000D92AC33B107D9F717E0ACE3B2E001C0B0
:100170001D92A132B107E1F711E0C6E4D1E004C05D
:100180002297FE010E94651AC434D107C9F70E9464
:10019000E3050C94621E0C940000DF92EF92FF9234
:1001A0000F931F93CF93DF9385E00E94FB140E946F
:1001B0008A0800E010E0DD24D39422C064E670E0F9
:1001C00080E090E00E9492089B01AC0180910D01BB
:1001D00090910E01A0910F01B091100128173907DD
:1001E0004A075B070CF4D8820894E108F1082296CC
:1001F000E114F10419F70F5F1F4F0E30110589F05C
:10020000C801880F991FEC0123E0CC0FDD1F2A9550
:10021000E1F7C80FD91FC35CDD4F89E0E82EF12C50
:10022000CDCFDF91CF911F910F91FF90EF90DF9095
:1002300008958F929F92AF92BF92CF92DF92EF92EA
:10024000FF920F931F93CF93DF93FC019B010196C5
:10025000CEE0D0E0BE010E94FF196C01C9010196F9
:1002600009E010E0B8010E94FF197C01CF010D9652
:10027000BE010E94FF195C01C9010896B8010E94E5
:10028000FF194F0163E0880C991C6A95E1F78E0E07
:100290009F1EF401EE0DFF1D6CE372E0EE0FFF1FD9
:1002A000E60FF71F0081F60143E0EE0FFF1F4A95AE
:1002B000E1F7EC0DFD1DEF01C20FD31FCC0FDD1FC9
:1002C000C60FD71F488150E0400F511DE501B3E034
:1002D000CC0FDD1FBA95E1F7CA0DDB1D2C0F3D1FBA
:1002E000220F331F260F371FD9012C91420F511DAA
:1002F000D401A80FB91FAA0FBB1FA60FB71F2C91BF
:10030000420F511DDF01AE0DBF1DAA0FBB1FA60F6F
:10031000B71F2C91420F511DDE01AE0DBF1DAA0F5C
:10032000BB1FA60FB71F2C91420F511DC80FD91F1D
:10033000CC0FDD1FC60FD71F2881420F511DE80FBC
:10034000F91FEE0FFF1FE60FF71F8081480F511DA9
:10035000CA01DF91CF911F910F91FF90EF90DF9035
:10036000CF90BF90AF909F908F900895DF92EF92C3
:10037000FF920F931F93CF93DF9380E00E94390485
:1003800085E00E94FB140E948A0800E010E0DD2452
:10039000D39425C064E670E080E090E00E9492086B
:1003A0009B01AC0180910D0190910E01A0910F0174
:1003B000B0911001281739074A075B0714F4D88257
:1003C00001C0188219820894E108F1082296E1140C
:1003D000F10401F70F5F1F4F0E30110589F0C801BE
:1003E000880F991FEC01E3E0CC0FDD1FEA95E1F7E0
:1003F000C80FD91FC45CDD4F79E0E72EF12CCACFBE
:10040000DF91CF911F910F91FF90EF90DF900895B2
:10041000CF92DF92EF92FF920F931F93CF93DF93D0
:1004200000E010E0DD24D39434C0C880C982C80144
:10043000B7010E94190120913803309139032F5FD1
:100440003F4F30933903209338038330910539F4BB
:10045000CC2029F4D982802F6E2D41E00BC0029769
:100460008230910548F08881813031F41982802FE3
:100470006E2D40E00E94AF020894E11CF11C229610
:1004800029E0E216F10489F60F5F1F4F0E301105C7
:1004900081F0C801880F991FEC0123E0CC0FDD1F0C
:1004A0002A95E1F7C80FD91FC45CDD4FEE24FF2465
:1004B000BCCF809138039091390301969093390312
:1004C0008093380323E18938920734F00E94CD00ED
:1004D000109239031092380380E090E00CC0418103
:1004E000408321503040329621153105C1F70196E5
:1004F0008E30910581F09C01220F331FF901A3E09A
:10050000EE0FFF1FAA95E1F7E20FF31FE45CFD4F2A
:1005100029E030E0E4CF66E970E080E090E00E94FE
:10052000F815DF91CF911F910F91FF90EF90DF9021
:10053000CF90089590913C0690FF10C091E0909369
:100540003D06882359F080913D06882339F061E00B
:1005500070E080E090E00E94F815F5CF0895EEE09D
:100560006E9FF0011124E80FF11DEE0FFF1FE95EF1
:10057000FE4F90818181880F8450292F26952695E2
:100580002695820F983010F028E101C020E0280F56
:10059000392F377081E090E0582F01C0550F3A9500
:1005A000EAF7352F442321F080913C0681FF47E094
:1005B000E0914006F0914106E20FF11DDF0180E07D
:1005C00090E050E0632F60958417950724F4208114
:1005D000232B208303C02C9126232C930196F09685
:1005E000D0968730910581F708950F931F93CF938D
:1005F000DF93082F162FC0E0D0E0802F6C2F412F03
:100600000E94AF022196C930D105B9F7DF91CF9191
:100610001F910F9108950F931F93CF93DF93082F8E
:10062000162FC0E0D0E08C2F602F412F0E94AF0228
:100630002196CE30D105B9F7DF91CF911F910F915F
:100640000895FF920F931F93CF93DF93F82E00E04E
:1006500010E00EC0802F6C2F4F2D0E94AF0221960C
:10066000C930D105B9F70F5F1F4F0E30110519F0D2
:10067000C0E0D0E0EFCFDF91CF911F910F91FF90BD
:1006800008952F923F924F925F926F927F928F9236
:100690009F92AF92BF92CF92DF92EF92FF920F9311
:1006A0001F93DF93CF93CDB7DEB72A970FB6F89499
:1006B000DEBF0FBECDBF682F70E080E090E00E94EB
:1006C000661720E030E04EEF52E40E94CD16C72EB0
:1006D000E82E092F762F272F3C2D4E2D502FCA01A3
:1006E000B9010E94181869877A871C0180EF8983F5
:1006F00022E0E22EF12CEC0EFD1E00E010E00F5F78
:100700001F4FB801882777FD8095982F0E946817A2
:1007100021EF3BE840EB50E40E94181820E030E065
:1007200040EC5FE30E947B1820E030E040E751E4BA
:100730000E9465169B01AC0160E070E08FE793E4D6
:100740000E9464160E943A17F70161937F010730F7
:100750001105A9F684EF96E00E94E00780916B06F0
:100760008823B9F4DE011196E0914306F091440626
:10077000CE0109962D912193209112012783A8176C
:10078000B907C1F706C061E070E080E090E00E9428
:10079000F815809142068823B1F7C0904506D090A5
:1007A00046068E010F5F1F4F760198E0492E512CAF
:1007B0004C0E5D1EBB24F801A1908F016A2D60953F
:1007C00070E0882777FD8095982F0E9468179B011D
:1007D000AC01B985AA856B2F7A2F822D932D0E94AB
:1007E00018183B014C016091130170E0882777FDD8
:1007F0008095982F0E9468179B01AC01C401B3013A
:100800000E9418189B01AC0160E070E08FE793E450
:100810000E9464160E943A17F70161937F0180914C
:10082000140187836A19B60E0415150521F6B094D4
:10083000F601B78280911201878781E0809342069A
:100840002A960FB6F894DEBF0FBECDBFCF91DF91D1
:100850001F910F91FF90EF90DF90CF90BF90AF90DE
:100860009F908F907F906F905F904F903F902F90D0
:1008700008951F93182F8091150161E00E94721452
:100880008091150160E00E949614809170008E7F27
:10089000809370008091B0008C7F8093B000809135
:1008A000B100877F8093B1008091B6008F7D8093E7
:1008B000B600809170008D7F809370008091B100B0
:1008C00083608093B1008091B1008B7F8093B100F1
:1008D00026E030E030933B0320933A0310933C062C
:1008E00010923D062CE333E030933F0620933E0602
:1008F00010FF07C08CEB94E0909341068093400674
:1009000004C0309341062093400689E496E090931A
:10091000440680934306409690934606809345068E
:10092000109242068FE70E94410380E090E00E940F
:10093000210380E00E949A0280913A0390913B0348
:100940008093B200809170008160809370008091EC
:100950003C0680FD07C00AC061E070E080E090E0E6
:100960000E94F81580913D068823B1F781E08093BD
:100970006B061F9108951F920F920FB60F921124CC
:100980002F933F934F935F936F937F938F939F9397
:10099000AF93BF93CF93DF93EF93FF931AB814B83D
:1009A0008091150161E00E94961460916906862F7E
:1009B00090E0E0914306F0914406E80FF91F20858E
:1009C0002093B10020812093B200673008F09BC0D3
:1009D00070916A067630D0F4272F30E0F901EE0FDF
:1009E000FF1F40913E0650913F06A0E3B0E08A9F72
:1009F000E0018B9FD00D9A9FD00D1124DE01AE0F28
:100A0000BF1FA40FB51F2E5F3F4F4CC07C3078F541
:100A1000272F30E0F901EE0FFF1F40913E06509165
:100A20003F06A0E3B0E08A9FE0018B9FD00D9A9F24
:100A3000D00D1124DE01AE0FBF1FA40FB51F8C9186
:100A40008AB98C918BB93196EC0FFD1FE40FF51F1D
:100A50002650304081E090E002C0880F991F2A950F
:100A6000E2F72081282B24B9808185B94EC0272F39
:100A700030E040913E0650913F06723138F5F90161
:100A8000EE0FFF1FA0E3B0E08A9FE0018B9FD00D27
:100A90009A9FD00D1124DE01AE0FBF1FA40FB51F0A
:100AA0002A50304081E090E002C0880F991F2A95BB
:100AB000E2F72C91282B2AB98C918BB93196EC0F47
:100AC000FD1FE40FF51F808184B9CECFF901EE0F31
:100AD000FF1FA0E3B0E08A9FE0018B9FD00D9A9F9B
:100AE000D00D1124DE01AE0FBF1FA40FB51F8C91D6
:100AF0008AB98C918BB93196EC0FFD1FE40FF51F6D
:100B000022513040A7CF1AB814B86F5F60936906BE
:100B1000683038F01092690680916A068F5F809382
:100B20006A0680916A068931B0F110926A06809156
:100B30003D068823B1F080913C0680FF12C01092E0
:100B40003D0680913E0690913F06209140063091EF
:100B5000410630933F0620933E06909341068093D2
:100B60004006809142068823B1F01092420680919F
:100B7000430690914406909348068093470620913F
:100B800045063091460630934406209343069093E1
:100B90004606809345068091150160E00E949614F8
:100BA000FF91EF91DF91CF91BF91AF919F918F9185
:100BB0007F916F915F914F913F912F910F900FBE59
:100BC0000F901F901895CF93DF930E9429160E94D3
:100BD000B601C3EDD6E00E9408022097E1F30E941F
:100BE000D306F9CFFC0184859585FC01E05CFF4FBD
:100BF000208131818E5B9F4FFC0180819181281B78
:100C0000390B2F733070C9010895FC0184859585D7
:100C1000FC01E05CFF4F40815181FC01EE5BFF4F26
:100C2000208131814217530741F00190F081E02D7E
:100C3000E80FF91F208130E002C02FEF3FEFC9011C
:100C40000895FC0184859585FC01E05CFF4F40819F
:100C50005181FC01EE5BFF4F208131814217530728
:100C600071F0A081B181A80FB91F2C918081918171
:100C700001968F7390709183808330E002C02FEFD4
:100C80003FEFC9010895DC011E968D919C911F973D
:100C9000FC01E05CFF4F8E5B9F4F40815181DC0186
:100CA0002D913C91119742175307B9F708951F935F
:100CB000FC01162F26853785D901A05CBF4F8D9189
:100CC0009C91019660E470E00E94FF19D901AE5B2F
:100CD000BF4F4D915C91119784179507D1F3D901BE
:100CE000A05CBF4F0D90BC91A02DA20FB31F1C9311
:100CF000A685B785A05CBF4F11969C938E93A6895D
:100D0000B7892C9181E090E0058C02C0880F991F73
:100D10000A94E2F7282B2C9381E090E01F9108952C
:100D2000FB01E05CFF4F208131812F5F3F4F2F732C
:100D30003070DB01AE5BBF4F4D915C911197241772
:100D4000350739F0A081B181A60FB71F8C9331838D
:100D50002083089508951F920F920FB60F921124C9
:100D60002F933F934F935F936F937F938F939F93B3
:100D7000AF93BF93EF93FF938091C6006CE676E04C
:100D80000E949006FF91EF91BF91AF919F918F913B
:100D90007F916F915F914F913F912F910F900FBE77
:100DA0000F901F90189584EF96E00E94F20500972F
:100DB00011F00E94AA0608951F920F920FB60F928B
:100DC00011242F933F935F936F937F938F939F9300
:100DD000AF93BF93EF93FF932091F0063091F1060C
:100DE0008091F2069091F3062817390731F480912B
:100DF000C1008F7D8093C10016C0E091F206F09192
:100E0000F306E055F94F20818091F2069091F306A8
:100E1000019660E470E00E94FF199093F3068093BE
:100E2000F2062093C600FF91EF91BF91AF919F9181
:100E30008F917F916F915F913F912F910F900FBE96
:100E40000F901F9018958F92AF92BF92CF92DF9222
:100E5000EF92FF920F931F93DF93CF93CDB7DEB73F
:100E6000FC011382128288EE93E0A0E0B0E084835C
:100E70009583A683B78387E192E09183808375870A
:100E8000648757874687318B208B138B028BF58ABB
:100E9000E48AD78AC68AB18EA08E828E8E85838F91
:100EA0008F85848F8889858F8989868FCF91DF91FF
:100EB0001F910F91FF90EF90DF90CF90BF90AF9078
:100EC0008F900895DF92EF92FF920F931F93CF932D
:100ED000DF93EC017A018B01DD24D394403081EE65
:100EE000580780E0680780E0780749F4DD24EC8942
:100EF000FD89108260E874E88EE190E00FC0EC8913
:100F0000FD8981E090E00E8C02C0880F991F0A9441
:100F1000E2F7808360E079E08DE390E0A80197013B
:100F20000E94121A2150304040405040569547953B
:100F30003795279580E12030380710F0DD20B1F695
:100F4000E889F9893083EA89FB892083EE89FF8962
:100F5000408181E090E09C010A8C02C0220F331F87
:100F60000A94E2F7422B4083EE89FF8940819C017D
:100F70000B8C02C0220F331F0A94E2F7422B4083EE
:100F8000EE89FF8940819C010C8C02C0220F331F27
:100F90000A94E2F7422B4083EE89FF8920810D8C71
:100FA00002C0880F991F0A94E2F7809582238083FC
:100FB000DF91CF911F910F91FF90EF90DF900895F7
:100FC000CF93DF93FC0186859785DC01A05CBF4F42
:100FD0008E5B9F4F4D915C911197EC012881398177
:100FE00042175307B9F7A689B7894C9181E090E081
:100FF0009C01028C02C0220F331F0A94E2F7209555
:1010000024232C93A689B7894C919C01038C02C0A0
:10101000220F331F0A94E2F7209524232C93A689EC
:10102000B7894C919C01048C02C0220F331F0A9493
:10103000E2F7209524232C93A689B7892C91058C5F
:1010400002C0880F991F0A94E2F7809582238C933F
:1010500084859585FC01EE5BFF4F20813181805CAA
:101060009F4FFC0131832083DF91CF91089510922F
:10107000F7061092F60688EE93E0A0E0B0E08093C9
:10108000F8069093F906A093FA06B093FB06E6EFF4
:10109000F6E087E192E0929382938CE696E0958762
:1010A000848780EB96E09787868785EC90E0918B2C
:1010B000808B84EC90E0938B828B80EC90E0958B1E
:1010C000848B81EC90E0978B868B86EC90E0918FFF
:1010D000808F84E0828F83E0838F87E0848F85E038
:1010E000858F81E0868F08950E94691A08950E9475
:1010F000031B089521E030E0FC018081882311F07A
:1011000020E030E0C901089521E0FC01208308952A
:1011100008950895009729F0BC0180E090E00E94B6
:10112000E81B0895EF92FF920F931F937B018C01B0
:10113000611571058105910549F00E94E31BA80125
:1011400097010E94341A9B01AC0103C020E030E0FB
:10115000A901B901CA011F910F91FF90EF90089565
:10116000EF92FF920F931F937B018C01621773071D
:101170008407950764F4CA01B9016E197F09800BD1
:10118000910B0E949208E60EF71E081F191FB70167
:10119000C8011F910F91FF90EF9008952F923F92F9
:1011A0004F925F926F927F928F929F92AF92BF9277
:1011B000CF92DF92EF92FF920F931F93DF93CF9323
:1011C000CDB7DEB73B014C0119012A016D897E893B
:1011D0008F89988D6A197B098C099D09621A730A97
:1011E000840A950AA40193010E94E019E218F30809
:1011F00004091509A80197010E94341A2A0D3B1D04
:101200004C1D5D1DB901CA01CF91DF911F910F9156
:10121000FF90EF90DF90CF90BF90AF909F908F9016
:101220007F906F905F904F903F902F90089508951A
:1012300070E0382F20E0622B732BCB010895CF9202
:10124000DF92EF92FF920F931F93CF93DF936C0186
:101250007B018A01C0E0D0E00FC0D7016D917D0114
:10126000D601ED91FC910190F081E02DC601099528
:10127000C80FD91F015010400115110571F7CE019B
:10128000DF91CF911F910F91FF90EF90DF90CF9062
:101290000895DB010D900020E9F7AD014150504069
:1012A000461B570BDC01ED91FC910280F381E02D90
:1012B00009950895EF92FF920F931F93CF93DF93B9
:1012C0007C01062F172FC0E0D0E0F8010F5F1F4F01
:1012D0006491662351F0F701A081B181ED91FC91F9
:1012E000C7010995C80FD91FF0CFCE01DF91CF916B
:1012F0001F910F91FF90EF900895AF92BF92CF9200
:10130000DF92EF92FF920F931F93CF93DF937C01B5
:101310006B01C0E0D0E000E010E010C0D701ED911B
:10132000FC91A080B180C601BE010E941711682FF8
:10133000C701F5010995080F191F2196F60184814F
:101340009581C817D90750F3C801DF91CF911F913C
:101350000F91FF90EF90DF90CF90BF90AF900895E6
:101360000E9449090895DC01ED91FC910190F08102
:10137000E02D099508959C01CB01DB01ED91FC91D5
:101380000190F081E02DB901099508950F931F9305
:10139000CF93DF93EC016DE00E94B3098C01CE0185
:1013A0006AE00E94B309080F191FC801DF91CF91AD
:1013B0001F910F9108950F931F93CF93DF93EC012B
:1013C0000E945A098C01CE010E94C609080F191FFC
:1013D000C801DF91CF911F910F9108950F931F9333
:1013E000CF93DF93EC010E947D098C01CE010E9416
:1013F000C609080F191FC801DF91CF911F910F91E6
:1014000008950F931F93CF93DF93EC010E94490936
:101410008C01CE010E94C609080F191FC801DF9177
:10142000CF911F910F9108950F931F93CF93DF9347
:10143000EC010E94B3098C01CE010E94C609080F7D
:10144000191FC801DF91CF911F910F9108950F933C
:101450001F93CF93DF93EC010E94BB098C01CE0157
:101460000E94C609080F191FC801DF91CF911F9173
:101470000F9108958F929F92AF92BF92CF92DF9279
:10148000EF92FF920F931F93DF93CF93CDB7DEB709
:10149000A1970FB6F894DEBF0FBECDBF6C01042F2D
:1014A000E52FCB01122F19A2223008F41AE021E215
:1014B000E22EF12CEC0EFD1E812E9924AA24BB24D1
:1014C00003C0022FE32FCA01602F7E2FA5019401D4
:1014D0000E94121A129F802D1124081B0894E10803
:1014E000F1080A3014F4005D01C0095CF7010083C3
:1014F000211531054105510521F7C601B7010E94AB
:101500004909A1960FB6F894DEBF0FBECDBFCF91AB
:10151000DF911F910F91FF90EF90DF90CF90BF90E0
:10152000AF909F908F9008952115310549F4DC010B
:10153000ED91FC910190F081E02D642F09950895C3
:101540000E943A0A08950F931F93CF93DF93EC0103
:101550000E94940A8C01CE010E94C609080F191F2F
:10156000C801DF91CF911F910F9108959A01AB01AE
:1015700060E070E00E94940A08950F931F93CF9348
:10158000DF93EC019A01AB0160E070E00E94940AE5
:101590008C01CE010E94C609080F191FC801DF91F6
:1015A000CF911F910F9108959A01462F50E060E06E
:1015B00070E00E94940A08950F931F93CF93DF93D6
:1015C000EC019A01462F50E060E070E00E94940A1E
:1015D0008C01CE010E94C609080F191FC801DF91B6
:1015E000CF911F910F910895CF92DF92EF92FF92CA
:1015F0000F931F93CF93DF93EC017A018B01211599
:10160000310541F4E881F9810190F081E02D642FEA
:1016100009951AC02A303105A9F477FF12C06DE28E
:101620000E94B3096C0144275527BA014E195F097E
:10163000600B710BCE012AE00E943A0AC80ED91E37
:1016400004C02AE00E943A0A6C01C601DF91CF91E2
:101650001F910F91FF90EF90DF90CF9008950F931F
:101660001F93CF93DF93EC010E94F40A8C01CE010B
:101670000E94C609080F191FC801DF91CF911F9161
:101680000F9108959A01FB01AF01662757FD609500
:10169000762F0E94F40A08950F931F93CF93DF9340
:1016A000EC019A01CB01AC01662757FD6095762FBE
:1016B000CE010E94F40A8C01CE010E94C609080FD7
:1016C000191FC801DF91CF911F910F9108956F925B
:1016D0007F929F92AF92BF92CF92DF92EF92FF9252
:1016E0000F931F93CF93DF933C017A018B01C22E9E
:1016F000CB01BA0120E030E0A9010E94C91687FFA2
:101700000AC0C3016DE20E94B309EC0117FB1095FA
:1017100017F9109502C0C0E0D0E0DD2450E040E0B1
:1017200030E02FE311C0DA01F9016B2F742F8F2FF6
:10173000922F20E030E040E251E40E94CD16562F77
:10174000472F382F292FD394DC1468F3C801B70131
:10175000DA01F9012B2F342F4F2F5E2F0E946516CF
:101760005B01F82E992E7B2D0E943A17162FD72E4B
:10177000E82E092F0E9466179B01AC016A2D7B2D74
:101780008F2D992D0E946416962EA72EB82EF92E15
:10179000C301412F5D2D6E2D702F2AE030E00E9495
:1017A000940AC80FD91FCC20B9F1C30160E071E0E1
:1017B0000E944909C80FD91F2FC0692D7A2D8B2D82
:1017C0009F2D20E030E040E251E40E941818D62E10
:1017D000B72EA82E992E0E9435177B010027F7FC03
:1017E0000095102FC301B801A7012AE030E00E9444
:1017F000F40AC80FD91FC801B7010E9468179B01DE
:10180000AC016D2D7B2D8A2D992D0E946416962E8C
:10181000A72EB82EF92ECA94CC2079F6CE01DF91EE
:10182000CF911F910F91FF90EF90DF90CF90BF90DD
:10183000AF909F907F906F9008950E94670B0895DE
:101840000F931F93CF93DF93EC010E94670B8C01E2
:10185000CE010E94C609080F191FC801DF91CF9160
:101860001F910F910895FC01808191810E94031BBB
:101870000895CF93DF93EC0188819981009711F04F
:101880000E94031B198218821D821C821B821A82ED
:10189000DF91CF9108950F931F93CF93DF93EC01C6
:1018A0008B016F5F7F4F888199810E94F11B0097A8
:1018B00031F0998388831B830A8381E001C080E033
:1018C000DF91CF911F910F910895CF93DF93EC019A
:1018D00088819981009729F08A819B8186179707D3
:1018E00078F4CE010E944B0C882341F08C819D81BD
:1018F000009731F4E881F981108202C080E001C0D4
:1019000081E0DF91CF910895EF92FF920F931F93A3
:10191000CF93DF93EC017B018A01BA010E94650C31
:10192000882321F4CE010E94390C07C01D830C834B
:1019300088819981B7010E942A1DCE01DF91CF9144
:101940001F910F91FF90EF900895CF93DF93FC01CB
:1019500011821082138212821582148216826115FE
:10196000710559F0EB0109900020E9F7AE014150F3
:101970005040461B570B0E94840CDF91CF91089575
:10198000EF92FF92CF93DF93EC01FB01861797074D
:1019900061F0608171816115710529F04481558183
:1019A0000E94840C02C00E94390CCE01DF91CF91BD
:1019B000FF90EF900895FC01118210821382128231
:1019C0001582148216820E94C00C08950F931F93F3
:1019D0008C016115710561F0DB010D900020E9F7C4
:1019E000AD0141505040461B570B0E94840C02C071
:1019F0000E94390CC8011F910F910895EF92FF9238
:101A00000F931F93DF93CF93CDB7DEB7A1970FB698
:101A1000F894DEBF0FBECDBF7C01CB01BA01F70148
:101A200011821082138212821582148216828E0114
:101A30000F5F1F4FA80130E00E94DD1DC701B801F4
:101A40000E94E60CA1960FB6F894DEBF0FBECDBF84
:101A5000CF91DF911F910F91FF90EF900895EF923A
:101A6000FF920F931F93DF93CF93CDB7DEB7A2976B
:101A70000FB6F894DEBF0FBECDBF7C01CB01BA011B
:101A8000F70111821082138212821582148216824B
:101A90008E010F5F1F4FA80130E00E94941DC70107
:101AA000B8010E94E60CA2960FB6F894DEBF0FBEF6
:101AB000CDBFCF91DF911F910F91FF90EF900895CF
:101AC000EF92FF920F931F93DF93CF93CDB7DEB7C3
:101AD00061970FB6F894DEBF0FBECDBF7C01CB017E
:101AE000F7011182108213821282158214821682EB
:101AF0008E010F5F1F4FB80150E00E94021EC70108
:101B0000B8010E94E60C61960FB6F894DEBF0FBED6
:101B1000CDBFCF91DF911F910F91FF90EF9008956E
:101B2000EF92FF920F931F93DF93CF93CDB7DEB762
:101B300062970FB6F894DEBF0FBECDBF7C01CB011C
:101B4000F70111821082138212821582148216828A
:101B50008E010F5F1F4FB80150E00E94731DC70137
:101B6000B8010E94E60C62960FB6F894DEBF0FBE75
:101B7000CDBFCF91DF911F910F91FF90EF9008950E
:101B8000EF92FF920F931F93DF93CF93CDB7DEB702
:101B900029970FB6F894DEBF0FBECDBF7C01862F0C
:101BA000F70111821082138212821582148216822A
:101BB00090E08E010F5F1F4FB80150E00E94021E9F
:101BC000C701B8010E94E60C29960FB6F894DEBF53
:101BD0000FBECDBFCF91DF911F910F91FF90EF907E
:101BE0000895DF93CF9300D0CDB7DEB7FC0111820B
:101BF00010821382128215821482168269831A82DD
:101C0000BE016F5F7F4F0E94E60C0F900F90CF9147
:101C1000DF910895EF92FF920F931F93CF93DF937D
:101C2000EC017B010C811D8161157105B9F0411535
:101C3000510591F0040F151FB8010E94650C88230F
:101C400069F0288139818C819D81820F931FB701B2
:101C50000E942A1D1D830C8381E001C080E0DF917A
:101C6000CF911F910F91FF90EF900895FB0160813C
:101C70007181448155810E940A0E08956115710594
:101C800061F0DB010D900020E9F7AD0141505040BB
:101C9000461B570B0E940A0E089580E00895DF93BB
:101CA000CF9300D0CDB7DEB769831A82BE016F5FD4
:101CB0007F4F41E050E00E940A0E0F900F90CF91AD
:101CC000DF910895EF92FF920F931F93DF93CF93CD
:101CD00000D000D0CDB7DEB77C01862F90E08E011A
:101CE0000F5F1F4FB8014AE050E00E94731DF801DA
:101CF00001900020E9F7AF0141505040401B510BCB
:101D0000C701B8010E940A0E0F900F900F900F901C
:101D1000CF91DF911F910F91FF90EF900895EF9277
:101D2000FF920F931F93DF93CF93CDB7DEB7279723
:101D30000FB6F894DEBF0FBECDBF7C01CB018E0184
:101D40000F5F1F4FB8014AE050E00E94731DF80179
:101D500001900020E9F7AF0141505040401B510B6A
:101D6000C701B8010E940A0E27960FB6F894DEBF8D
:101D70000FBECDBFCF91DF911F910F91FF90EF90DC
:101D80000895EF92FF920F931F93DF93CF9300D0AC
:101D900000D000D0CDB7DEB77C01CB018E010F5F44
:101DA0001F4FB8014AE050E00E94021EF801019066
:101DB0000020E9F7AF0141505040401B510BC701D3
:101DC000B8010E940A0E26960FB6F894DEBF0FBE29
:101DD000CDBFCF91DF911F910F91FF90EF900895AC
:101DE000EF92FF920F931F93DF93CF93CDB7DEB7A0
:101DF0002C970FB6F894DEBF0FBECDBF7C01CB0190
:101E0000BA018E010F5F1F4FA8012AE030E00E9447
:101E1000941DF80101900020E9F7AF0141505040B6
:101E2000401B510BC701B8010E940A0E2C960FB639
:101E3000F894DEBF0FBECDBFCF91DF911F910F9100
:101E4000FF90EF900895EF92FF920F931F93DF930F
:101E5000CF93CDB7DEB72B970FB6F894DEBF0FBE8A
:101E6000CDBF7C01CB01BA018E010F5F1F4FA801CE
:101E70002AE030E00E94DD1DF80101900020E9F722
:101E8000AF0141505040401B510BC701B8010E94A7
:101E90000A0E2B960FB6F894DEBF0FBECDBFCF91C2
:101EA000DF911F910F91FF90EF9008950F931F9373
:101EB0008C01FB0160817181448155810E940A0E71
:101EC000882319F4C8010E94390CC8011F910F9191
:101ED00008950F931F938C016115710569F0DB0163
:101EE0000D900020E9F7AD0141505040461B570BC3
:101EF0000E940A0E882319F4C8010E94390CC801F7
:101F00001F910F9108950F931F938C010E944F0E04
:101F1000882319F4C8010E94390CC8011F910F9140
:101F200008950F931F938C010E94620E882319F469
:101F3000C8010E94390CC8011F910F9108950F9399
:101F40001F938C010E948F0E882319F4C8010E94F0
:101F5000390CC8011F910F9108950F931F938C01A5
:101F60000E94C10E882319F4C8010E94390CC801CF
:101F70001F910F9108950F931F938C010E94F00EF3
:101F8000882319F4C8010E94390CC8011F910F91D0
:101F900008950F931F938C010E94230F882319F437
:101FA000C8010E94390CC8011F910F910895CF9369
:101FB000DF93FC01DB0180819181009731F06D910D
:101FC0007C91119761157105E9F4CD91DC91119720
:101FD000209769F014962D913C91159721153105A4
:101FE00031F0288130E0309521953F4F12C00097A5
:101FF00071F0248135812115310549F0FC012081E2
:1020000030E007C00E94211D282F392F02C020E098
:1020100030E0C901DF91CF910895FC0144815581E1
:10202000FB01248135814217530729F40E94D70F01
:1020300021E0009709F020E0822F0895FC018481BF
:102040009581009741F46115710519F081E0FB015C
:1020500009C081E008950190F081E02D61157105BE
:1020600031F481E09081992359F080E00895CF0107
:102070000E94211D9C0181E02115310509F080E0BD
:1020800008950E94D70F892F881F8827881F0895D9
:102090000E94D70F21E0181619060CF020E0822FBD
:1020A00008950E94D70F21E0181619060CF420E0BD
:1020B000822F08950E94D70F892F8095881F882727
:1020C000881F0895EF92FF920F931F93CF93DF9392
:1020D000FC01DB018617970729F18481958114960D
:1020E0002D913C91159782179307F1F40097D1F049
:1020F00000811181CD91DC9111970FC0992787FD47
:1021000090950E94EB1C7C018991992787FD909501
:102110000E94EB1CE816F90639F4F80181918F0151
:10212000882361F781E001C080E0DF91CF911F91AA
:102130000F91FF90EF900895FC01DB01CA01149606
:102140004D915C91159724813581241B350B2817FF
:102150003907A0F0208131812115310579F06D9189
:102160007C9111976115710559F0820F931F0E94A0
:10217000311D9C0181E02115310519F080E00895A1
:1021800080E00895FC0144815581FB012481358163
:102190004217530728F040E050E00E949C10089539
:1021A00080E00895FC01DB018481958114964D91B6
:1021B0005C91159784179507B0F020813181211526
:1021C000310589F06D917C9111976115710569F068
:1021D000841B950B820F931F0E94211D9C0181E09F
:1021E0002115310519F080E0089580E00895FC0183
:1021F000848195816817790730F40190F081E02D92
:10220000E60FF71F40830895FC01848195816817CC
:10221000790720F480819181009729F410921307A7
:1022200063E177E002C0680F791FCB010895FC01DC
:10223000848195816817790748F48081918100979E
:1022400039F0680F791FFB018081089580E00895BF
:1022500080E008950E94171108950F931F93CF9364
:10226000DF93FC018B0141155105F1F061157105FA
:10227000D9F0C481D5812C173D0718F0FB011082DD
:1022800013C041505040C21BD30B4C175D0708F4DC
:10229000EA0160817181620F731FC801AE010E9463
:1022A0003F1DC00FD11F1882DF91CF911F910F9159
:1022B0000895CF93DF93FC01CA0124813581421731
:1022C000530778F4C081D181772767FD70958C0F13
:1022D0009D1F0E94161D009721F09C012C1B3D0B99
:1022E00002C02FEF3FEFC901DF91CF91089540E089
:1022F00050E00E9459110895CF93DF93FC01CA0169
:10230000248135814217530778F4C081D181FB01C4
:10231000608171818C0F9D1F0E94591D009721F0D3
:102320009C012C1B3D0B02C02FEF3FEFC901DF9139
:10233000CF91089540E050E00E947C110895DF9213
:10234000EF92FF920F931F93CF93DF93EC018C8159
:102350009D8148175907F8F47A010894E11CF11C93
:10236000E881F981EE0DFF1DD0801082088119816E
:10237000772767FD7095C8010E944E1D0E0D1F1D29
:10238000F801D082009739F028813981AC01421BD5
:10239000530B9A0102C02FEF3FEFC901DF91CF919C
:1023A0001F910F91FF90EF90DF900895FC01448101
:1023B0005581415050400E949F110895AF92BF92A5
:1023C000CF92DF92EF92FF920F931F93CF93DF9301
:1023D000FC016B018A01DB0114962D913C9115974C
:1023E0002115310551F184819581009731F18217D2
:1023F000930718F14817590718F08C010150104045
:10240000E080F180C701CFEFDFEF5701A00EB11ED2
:1024100010C0F601608171810E94591D009779F00A
:102420009C012E193F090217130708F49E0101961B
:10243000E901A816B90668F702C0CFEFDFEFCE01B9
:10244000DF91CF911F910F91FF90EF90DF90CF9090
:10245000BF90AF900895FC0144815581FB01248118
:102460003581421B530B0E94DE110895AF92BF923B
:10247000CF92DF92EF92FF920F931F93CF93DF9350
:10248000F82EE92E6B018A01E9012417350748F47B
:10249000342F212F8E01C901A92EE5015E01B22E34
:1024A000E5018F2D9E2D62E071E00E94A50CD60102
:1024B00014968D919C91159780179107D8F08C17E1
:1024C0009D0708F4EC01D601ED91FC911197EC0FFA
:1024D000FD1FB08010826D917C91600F711F8F2D58
:1024E0009E2D0E94E60CD601ED91FC911197EC0F08
:1024F000FD1FB0828F2D9E2DDF91CF911F910F91E7
:10250000FF90EF90DF90CF90BF90AF900895CF9362
:10251000DF93EC01FB01248135810E943612CE014C
:10252000DF91CF910895DC01ED91FC9111973097E7
:1025300029F40895861709F4408331968081882311
:10254000C9F708952F923F924F925F926F927F92B8
:102550008F929F92AF92BF92CF92DF92EF92FF92B3
:102560000F931F93CF93DF937C012B016A01DC0152
:1025700014966D907C9015976114710409F4D9C07C
:10258000FB01848095808114910409F4D2C0DA01A2
:102590001496AD90BC901597A818B908FC0100815D
:1025A0001181A114B104F1F413C0D6016C911196FC
:1025B0007C91119714964D915C911597CE010E94D4
:1025C000FB1CD60114960D911C9115970C0F1D1F25
:1025D000F20160817181C8010E94591DEC010097D0
:1025E00021F7A7C0B7FC02C0E30142C048012DC0DB
:1025F000E301C01BD10BC401B801AE010E94FB1C5A
:10260000C80DD91DD6016C9111967C911197149625
:102610004D915C911597CE010E94FB1CD60114963A
:102620008D909C9015978C0E9D1EF2010481158152
:10263000060D171DD70114968D919C9115978A0D43
:102640009B1D15969C938E931497F2016081718166
:10265000C8010E94591D3C01009751F6C401B80100
:102660000E942A1D66C08C01080D191DCA0DDB1DB4
:10267000D2016D917C91C8010E94591D009799F774
:10268000C615D70509F455C0F701828193818C17CF
:102690009D0708F045C0C701BE010E944B0C88236E
:1026A00009F447C03DC0C701B201A9010E94DE1173
:1026B000EC0197FD3EC0D7016D917C911197F2011D
:1026C000848195818C0F9D1F680F791F14964D9101
:1026D0005C911597481B590BCB018A0D9B1D0E94DD
:1026E000041DD70114968D919C9115978A0D9B1D01
:1026F00015969C938E931497ED91FC911197E80F8A
:10270000F91F10822D913C912C0F3D1FF601608125
:10271000718144815581C9010E94FB1C9E0105C045
:10272000D70114962D913C9115972150304037FFD9
:10273000BACFDF91CF911F910F91FF90EF90DF9073
:10274000CF90BF90AF909F908F907F906F905F9051
:102750004F903F902F900895CF93DF93FC01C0815D
:10276000D181209739F409C0992787FD90950E945F
:10277000EB1C899388818823B9F7DF91CF91089565
:10278000CF93DF93FC01C081D181209739F409C038
:10279000992787FD90950E94F31C8993888188234F
:1027A000B9F7DF91CF910895AF92BF92CF92DF92A8
:1027B000EF92FF920F931F93CF93DF936C01DC0195
:1027C000ED90FC901197E114F10409F443C01496C4
:1027D000AD90BC901597A114B104E1F18701E80117
:1027E00088810F5F1F4F992787FD90950E94E31CFA
:1027F0000097A9F78501015010400E0D1F1DF8012B
:102800008081992787FD90950E94E31C009731F005
:102810000C171D0718F001501040F1CF0F5F1F4F2C
:102820000C1B1D0BD60115961C930E931497EC16DA
:10283000FD0628F4C701BE01A8010E94FB1CD601B9
:10284000ED91FC91119714968D919C911597E80F3D
:10285000F91F1082DF91CF911F910F91FF90EF90A0
:10286000DF90CF90BF90AF900895FC01808191815F
:10287000009729F00E94BC1C9B01AC0103C020E022
:1028800030E0A901B901CA010895833071F08430A4
:1028900028F48130A1F0823021F514C08630B1F0E7
:1028A0008730D1F08430E9F404C0809180008F77C4
:1028B00003C0809180008F7D80938000089584B54F
:1028C0008F7702C084B58F7D84BD08958091B0005C
:1028D0008F778093B00008958091B0008F7D8093B2
:1028E000B000089590E0FC01E45EFE4F2491FC01ED
:1028F000E85FFE4FE491EE23C1F0F0E0EE0FFF1F22
:10290000E651FF4F85919491DC01662341F49FB716
:10291000F8948C91209582238C939FBF08959FB744
:10292000F8948C91822B8C939FBF08950F931F93E3
:10293000DF93CF930F92CDB7DEB7282F30E0F901A8
:10294000E05DFE4F8491F901E45EFE4F1491285F33
:102950003E4FF90104910023D9F0882321F06983C7
:102960000E9445146981E02FF0E0EE0FFF1FEC504C
:10297000FF4F85919491DC019FB7F894662321F471
:102980008C911095812302C08C91812B8C939FBFD9
:102990000F90CF91DF911F910F9108950F931F9387
:1029A000282F30E0F901E05DFE4F8491F901E45EEB
:1029B000FE4F0491285F3E4FF9011491112391F0CD
:1029C000882311F00E944514E12FF0E0EE0FFF1F65
:1029D000E250FF4F85919491DC018C91802321E09E
:1029E00030E011F420E030E0C9011F910F9108950B
:1029F0008093160108958E3008F08E508770909164
:102A000016019295990F990F907C982B90937C00CA
:102A100080917A00806480937A0080917A0086FDAC
:102A2000FCCF2091780030917900932F80E030E046
:102A3000282B392BC90108951F93CF93DF93182FAB
:102A4000EB0161E00E947214209709F44AC0CF3F65
:102A5000D10509F449C0E12FF0E0E05DFE4FE491BB
:102A6000E330C1F0E43028F4E13051F0E230B1F568
:102A70000CC0E63019F1E73049F1E43079F514C0C3
:102A800084B5806884BDC7BD33C084B5806284BD11
:102A9000C8BD2EC080918000806880938000D09354
:102AA0008900C093880024C0809180008062809358
:102AB0008000D0938B00C0938A001AC08091B00030
:102AC00080688093B000C093B30012C08091B000C2
:102AD00080628093B000C093B4000AC0C038D105B2
:102AE0001CF4812F60E002C0812F61E00E949614E7
:102AF000DF91CF911F9108951F920F920FB60F9201
:102B000011242F933F938F939F93AF93BF93809103
:102B1000180790911907A0911A07B0911B073091DF
:102B20001C070196A11DB11D232F2D5F2D3720F00D
:102B30002D570196A11DB11D20931C0780931807E6
:102B400090931907A0931A07B0931B07809114075D
:102B500090911507A0911607B09117070196A11D36
:102B6000B11D8093140790931507A0931607B09397
:102B70001707BF91AF919F918F913F912F910F9028
:102B80000FBE0F901F9018958FB7F89420911807DB
:102B90003091190740911A0750911B078FBFB90157
:102BA000CA0108959FB7F894209114073091150732
:102BB000409116075091170786B5A89B06C08F3F16
:102BC00021F02F5F3F4F4F4F5F4F9FBF542F432F39
:102BD000322F2227280F311D411D511D82E0220F67
:102BE000331F441F551F8A95D1F7B901CA010895B3
:102BF000EF92FF920F931F93CF93DF937B018C0192
:102C00000E94D215EB010FC00E94D2156C1B7D0BE8
:102C100083E0683E780738F00894E108F10801097C
:102C20001109C851DC4FE114F1040105110561F7E8
:102C3000DF91CF911F910F91FF90EF900895019731
:102C400039F0880F991F880F991F02970197F1F7A4
:102C50000895789484B5826084BD84B5816084BD14
:102C600085B5826085BD85B5816085BDEEE6F0E005
:102C7000808181608083E1E8F0E010828081826061
:102C80008083808181608083E0E8F0E080818160E2
:102C90008083E1EBF0E0808184608083E0EBF0E012
:102CA000808181608083EAE7F0E0808184608083B6
:102CB0008081826080838081816080838081806860
:102CC00080831092C10008955058BB27AA270ED0C8
:102CD00075C166D130F06BD120F031F49F3F11F413
:102CE0001EF45BC10EF4E095E7FB51C1E92F77D1EB
:102CF00080F3BA17620773078407950718F071F419
:102D00009EF58FC10EF4E0950B2EBA2FA02D0B016E
:102D1000B90190010C01CA01A0011124FF27591B20
:102D200099F0593F50F4503E68F11A16F040A22F26
:102D3000232F342F4427585FF3CF46953795279597
:102D4000A795F0405395C9F77EF41F16BA0B620B96
:102D5000730B840BBAF09150A1F0FF0FBB1F661FDD
:102D6000771F881FC2F70EC0BA0F621F731F841F20
:102D700048F4879577956795B795F7959E3F08F046
:102D8000B3CF9395880F08F09927EE0F9795879505
:102D90000895D9D008F481E008950CD00FC107D16F
:102DA00040F0FED030F021F45F3F19F0F0C0511137
:102DB00039C1F3C014D198F39923C9F35523B1F362
:102DC000951B550BBB27AA2762177307840738F09A
:102DD0009F5F5F4F220F331F441FAA1FA9F333D0F9
:102DE0000E2E3AF0E0E830D091505040E695001CAD
:102DF000CAF729D0FE2F27D0660F771F881FBB1F69
:102E0000261737074807AB07B0E809F0BB0B802D42
:102E1000BF01FF2793585F4F2AF09E3F510568F08E
:102E2000B6C000C15F3FECF3983EDCF38695779522
:102E30006795B795F7959F5FC9F7880F911D969590
:102E4000879597F90895E1E0660F771F881FBB1FEC
:102E5000621773078407BA0720F0621B730B840B99
:102E6000BA0BEE1F88F7E095089504D06894B1116D
:102E7000D9C00895BCD088F09F5790F0B92F9927FA
:102E8000B751A0F0D1F0660F771F881F991F1AF075
:102E9000BA95C9F712C0B13081F0C3D0B1E008953E
:102EA000C0C0672F782F8827B85F39F0B93FCCF3BF
:102EB000869577956795B395D9F73EF4909580956B
:102EC000709561957F4F8F4F9F4F0895E89409C08B
:102ED00097FB3EF490958095709561957F4F8F4F4D
:102EE0009F4F9923A9F0F92F96E9BB279395F69563
:102EF000879577956795B795F111F8CFFAF4BB0FE1
:102F000011F460FF1BC06F5F7F4F8F4F9F4F16C044
:102F1000882311F096E911C0772321F09EE8872FCE
:102F2000762F05C0662371F096E8862F70E060E08A
:102F30002AF09A95660F771F881FDAF7880F969503
:102F4000879597F90895990F0008550FAA0BE0E8A7
:102F5000FEEF16161706E807F907C0F0121613065B
:102F6000E407F50798F0621B730B840B950B39F49B
:102F70000A2661F0232B242B252B21F408950A2601
:102F800009F4A140A6958FEF811D811D089597F941
:102F90009F6780E870E060E008959FEF80EC0895FF
:102FA00000240A9416161706180609060895002428
:102FB0000A9412161306140605060895092E0394A2
:102FC000000C11F4882352F0BB0F40F4BF2B11F416
:102FD00060FF04C06F5F7F4F8F4F9F4F089557FD75
:102FE0009058440F551F59F05F3F71F04795880F77
:102FF00097FB991F61F09F3F79F08795089512160E
:1030000013061406551FF2CF4695F1DF08C01616B9
:1030100017061806991FF1CF86957105610508946A
:103020000895E894BB2766277727CB0197F9089581
:103030000BD0C4CFB5DF28F0BADF18F0952309F024
:10304000A6CFABCF1124EECFCADFA0F3959FD1F36B
:10305000950F50E0551F629FF001729FBB27F00D46
:10306000B11D639FAA27F00DB11DAA1F649F66279B
:10307000B00DA11D661F829F2227B00DA11D621FEA
:10308000739FB00DA11D621F839FA00D611D221FA4
:10309000749F3327A00D611D231F849F600D211D88
:1030A000822F762F6A2F11249F5750408AF0E1F02B
:1030B00088234AF0EE0FFF1FBB1F661F771F881F74
:1030C00091505040A9F79E3F510570F060CFAACFB4
:1030D0005F3FECF3983EDCF3869577956795B7955F
:1030E000F795E7959F5FC1F7FE2B880F911D969589
:1030F000879597F90895FA01EE0FFF1F3096210585
:10310000310599F16115710561F48038BFE39B07C2
:1031100049F168949038810561F08038BFEF9B07D2
:1031200041F0992342F5FF3FE1053105210511F1F9
:10313000E8940894E795D901AA2329F4AB2FBE2F70
:10314000F85FD0F310C0FF5F70F4A695E0F7F73991
:1031500050F019F0FF3A38F49F779F930CD00F90FE
:1031600007FC905808953EF018CF60E070E080E8CA
:103170009FE308954FE79F775F934F933F932F937C
:103180009ED02F913F914F915F9152DF05C019F46E
:103190000EF0FDCE46CF01CF2ADFC8F39638C0F738
:1031A00007F80F92E8942BE33AEA48EB5FE74EDF2B
:1031B0000F920F920F924DB75EB70F92C0D0E8E614
:1031C000F0E016D04F915F91EF91FF91E595EE1FE2
:1031D000FF1F49F0FE57E0684427EE0F441FFA95A1
:1031E000E1F74195550B32D00F9007FE26C00895A8
:1031F000DF93CF931F930F93FF92EF92DF927B01A8
:103200008C01689405C0DA2EEF011EDFFE01E89400
:10321000A5912591359145915591AEF3EF0166DD6C
:10322000FE019701A801DA9479F7DF90EF90FF9003
:103230000F911F91CF91DF9108959B01AC0160E048
:1032400070E080E89FE3A9CDA2CEACC0D0DEE8F369
:103250009923D9F3940F511DBBF39150504094F032
:1032600059F0882332F0660F771F881F9150504025
:10327000C1F79E3F510544F7880F911D969587959C
:1032800097F908955F3FACF0983E9CF0BB27869578
:1032900077956795B79508F4B1609395C1F7BB0F23
:1032A00058F711F460FFE8CF6F5F7F4F8F4F9F4F4C
:1032B000E3CFB8CE0EF076C070CE689468CE97DEBD
:1032C000C8F39923D1F3C6F3DF93CF931F930F93E2
:1032D000FF92C92FDD2788232AF02197660F771FD9
:1032E000881FDAF720E030E040E85FEB9FE38839A1
:1032F00020F0803E30F021968F77E7DCE0E9F0E0C7
:1033000003C0E3DCEDEBF0E073DF8B01BE01EC0109
:10331000FB2E6F5771097595771F880B990BD8DDB8
:1033200028E132E741E35FE38FDEAF2D9801AE0184
:10333000FF900F911F91CF91DF91D8DC3FCEFA0122
:10334000DC01AA0FBB1F9B01AC01BF5728F4222749
:103350003327442750781FC0B75188F4AB2F00247F
:10336000469537952795011CA395D2F3002069F067
:10337000220F331F441FB395DAF30DD0A5CC613073
:103380007105A0E88A07B94630F49B01AC016627B5
:10339000772788279078309621F0208331834283E5
:1033A000538308959F3F31F0915020F4879577958E
:1033B0006795B795880F911D9695879597F908950C
:1033C000629FD001739FF001829FE00DF11D649F09
:1033D000E00DF11D929FF00D839FF00D749FF00D95
:1033E000659FF00D9927729FB00DE11DF91F639F36
:1033F000B00DE11DF91FBD01CF011124089597FB08
:10340000092E07260AD077FD04D049D006D0002027
:103410001AF4709561957F4F0895F6F79095819510
:103420009F4F0895A1E21A2EAA1BBB1BFD010DC0E0
:10343000AA1FBB1FEE1FFF1FA217B307E407F50764
:1034400020F0A21BB30BE40BF50B661F771F881F40
:10345000991F1A9469F760957095809590959B01D6
:10346000AC01BD01CF01089597FB092E05260ED0B2
:1034700057FD04D0D7DF0AD0001C38F45095409592
:10348000309521953F4F4F4F5F4F0895F6F7909538
:103490008095709561957F4F8F4F9F4F0895AA1B20
:1034A000BB1B51E107C0AA1FBB1FA617B70710F02F
:1034B000A61BB70B881F991F5A95A9F78095909561
:1034C000BC01CD010895EE0FFF1F0590F491E02D92
:1034D0000994CF93DF938230910510F482E090E05D
:1034E000E0911F07F091200740E050E020E030E03D
:1034F00026C06081718168177907E0F06817790745
:1035000081F4828193812115310531F0D90113961F
:103510009C938E9312972BC09093200780931F0744
:1035200026C04115510519F06417750718F4AB0151
:10353000E901DF019F0172816381E72FF62F309748
:10354000C1F64115510501F1481B590B4430510595
:1035500080F412968D919C911397209719F09B837C
:103560008A8304C09093200780931F07FD01329641
:1035700046C0FD01E40FF51F8193919342505040E6
:1035800011965C934E933BC020911D0730911E070E
:103590002115310541F42091050130910601309348
:1035A0001E0720931D072091070130910801211566
:1035B000310541F42DB73EB740910301509104010C
:1035C000241B350BE0911D07F0911E07E217F3074E
:1035D000A0F42E1B3F0B2817390778F0AC014E5F83
:1035E0005F4F2417350748F04E0F5F1F50931E079B
:1035F00040931D078193919302C0E0E0F0E0CF017A
:10360000DF91CF910895CF93DF93009709F491C094
:10361000FC0132971382128260911F07709120077C
:103620006115710581F420813181280F391F809146
:103630001D0790911E078217930799F5F0931E07B7
:10364000E0931D0776C0DB0180E090E002C0CD0171
:10365000D901AE17BF0748F412962D913C911397EC
:1036600021153105A1F7CD0121C0B383A283EF015C
:10367000499159919E01240F351FA217B30779F480
:103680002D913C911197240F351F2E5F3F4F3183B1
:10369000208312962D913C911397338322830097B8
:1036A00029F4F0932007E0931F0743C0DC01139631
:1036B000FC93EE9312974D915D91A40FB51FEA17FD
:1036C000FB0769F420813181240F351F2E5F3F4FA6
:1036D000EC0139832883228133813B832A83E0E014
:1036E000F0E002C0FB01BC01DB0112968D919C91C0
:1036F00013970097B9F79B012E5F3F4F8D919C91D7
:103700001197820F931F40911D0750911E07481774
:10371000590779F4309729F41092200710921F0767
:1037200002C0138212822250304030931E07209331
:103730001D07DF91CF910895A0E0B0E0E2EAFBE140
:103740000C94331EEC01688179818A819B8161151B
:1037500071058105910521F464E279ED8BE597E02F
:103760002DE133EF41E050E00E94341A79018A01E3
:1037700027EA31E440E050E00E94E0195B016C016F
:10378000C801B7012CEE34EF4FEF5FEF0E94E01954
:103790009B01AC012A0D3B1D4C1D5D1D57FF04C054
:1037A0002150304040405048288339834A835B830E
:1037B0005F77B901CA01CDB7DEB7EAE00C944F1EBE
:1037C0000E949C1B089589E091E00E949C1B089533
:1037D0006093090170930A0180930B0190930C018F
:1037E0000895A0E0B0E0E7EFFBE10C94311E8C01FE
:1037F000CB010115110529F40E94691A082F192F10
:10380000B5C0D80112979801260F371F2A173B071A
:1038100008F4AAC0ED90FC901197E616F706D0F0D8
:1038200045E0E416F10408F4A1C0A701445050405B
:103830004617570708F49AC0A70142505040461B4C
:10384000570BF901419351936D937C93CF010E94E3
:10385000031B8CC05B01AE18BF0848018E0C9F1C77
:10386000E0911F07F0912007CC24DD24C0E0D0E0D8
:1038700041C0E815F90599F560817181AB014E5F92
:103880005F4F4A155B0558F1AB014A195B09CC241F
:10389000DD246894C1F8C40ED51E8280A380E5E0C3
:1038A000CE16D10448F0F9018282A382518340836D
:1038B00011969C938E9309C0C7010296860F971F9D
:1038C00011969C938E93E82DFA2D209719F0FB8387
:1038D000EA834CC0F0932007E0931F0747C0408164
:1038E0005181C416D50608F46A01EF015281438163
:1038F000E52FF42F309709F0BCCF40911D07509170
:103900001E0748155905E9F4C816D906D0F44091A8
:103910000701509108014115510541F44DB75EB7BB
:103920006091030170910401461B570B2417350762
:10393000D8F430931E0720931D0711969C938E9305
:1039400015C00E94691AC82EE6016E01D92EE60143
:10395000209751F08C2DB801A7010E94FB1CC801D3
:103960000E94031B860102C000E010E0C801CDB731
:10397000DEB7ECE00C944D1E1F93FC0199278827BD
:10398000BC01E89411911032E9F3193010F01E30A7
:10399000C8F31B3251F01D3249F4689406C00E94EE
:1039A000C81D610F711D811D911D119110531A3099
:1039B000B0F33EF490958095709561957F4F8F4F51
:1039C0009F4F1F910895911133C1803219F0895092
:1039D0008550D0F708959111089581548A5108F4C3
:1039E000805E855A08959111089581568A5108F490
:1039F000805285580895FB01DC0102C001900D92B0
:103A000041505040D8F708956817790768F4FB01D2
:103A1000DC01E40FF51FA40FB51F02C002900E9247
:103A200041505040D8F708950C94FB1CFC01819143
:103A3000861721F08823D9F7992708953197CF0168
:103A40000895FB01DC018D91019080190110D9F3DB
:103A5000990B0895FB01DC0101900D920020E1F724
:103A60000895FB01DC014150504030F08D910190F0
:103A7000801919F40020B9F7881B990B0895FB01F0
:103A8000DC014150504048F001900D920020C9F7F0
:103A900001C01D9241505040E0F70895FC0181E0C3
:103AA00090E00190061609F4CF010020D1F70197AC
:103AB0000895FB0151915523A9F0BF01DC014D91FF
:103AC00045174111E1F759F4CD010190002049F06B
:103AD0004D9140154111C9F3FB014111EFCF81E038
:103AE00090E001970895FB019F01E8944230C4F0F3
:103AF0004532B4F44A3029F497FB1EF49095819531
:103B00009F4F642F77270E944F1A805D8A330CF0F5
:103B1000895D8193CB010097A1F716F45DE2519383
:103B20001082C9010C941B1EFA01CF93FF93EF93EF
:103B3000223044F1253234F5C22FE894CA3049F4DA
:103B400097FB3EF490958095709561957F4F8F4FD0
:103B50009F4F2C2F332744275527FF93EF930E9425
:103B6000121AEF91FF91605D6A330CF0695D619309
:103B7000B901CA01605070408040904051F716F47E
:103B8000CDE2C19310828F919F91CF910C941B1E17
:103B9000592F482F372F262F660F771F881F991F01
:103BA000660F771F881F991F620F731F841F951F51
:103BB000660F771F881F991F0895FA01CF93FF930F
:103BC000EF932230CCF02532BCF4C22F2C2F3327B8
:103BD00044275527FF93EF930E94121AEF91FF910C
:103BE000605D6A330CF0695D6193B901CA01605090
:103BF00070408040904051F710828F919F91CF91FB
:103C00000C941B1EFB019F01423074F0453264F49A
:103C1000642F77270E944F1A805D8A330CF0895DEC
:103C20008193CB010097A1F71082C9010C941B1E50
:103C3000992788270895DC01FC01672F719177236C
:103C4000E1F7329704C07C916D9370836291AE1757
:103C5000BF07C8F308952F923F924F925F926F92E1
:103C60007F928F929F92AF92BF92CF92DF92EF920C
:103C7000FF920F931F93CF93DF93CDB7DEB7CA1B8D
:103C8000DB0B0FB6F894DEBF0FBECDBF09942A88B8
:103C9000398848885F846E847D848C849B84AA8460
:103CA000B984C884DF80EE80FD800C811B81AA81ED
:103CB000B981CE0FD11D0FB6F894DEBF0FBECDBFB8
:083CC000ED010895F894FFCF17
:103CC8002E00002000210700000100000032000043
:103CD800000103040213010D050D060D070D080D63
:103CE800090D0A0D0B0D0C0D04040D0D03030D0D2C
:103CF80002020D0C050C060C070C080C090C0A0C2A
:103D08000B0C0D0C04040C0C03030C0C02020C0B22
:103D1800050B060B070B080B090B0A0B0C0B0D0BFD
:103D280004040B0B03030B0B02020B0A050A060A19
:103D3800070A080A090A0B0A0C0A0D0A04040A0AE7
:103D480003030A0A02020A090509060907090809FC
:103D58000A090B090C090D090404090903030909D7
:103D68000202090805080608070809080A080B08D6
:103D78000C080D08040408080303080802020807D1
:103D880005070607080709070A070B070C070D07A9
:103D980004040707030307070202070605060706C8
:103DA800080609060A060B060C060D060404060694
:103DB80003030606020206050605070508050905A8
:103DC8000A050B050C050D05040405050303050587
:103DD8000202050000000057061F09F2052106052A
:103DE8000643060000000089081F09890889088918
:0C3DF8000889080000000089081F09006D
:00000001FF
